:020000040000FA
:1000000083160313810170298B138B1B0428AD0009
:10001000030EAE0083010A08AF008A0183130408AF
:10002000B0008B1834280B1826288C1A18288C2816
:100030001A08AA008C1E1F281A08AB0029142714BE
:10004000831603138C12831203138C28861F8828AF
:100050008B115030B100B10B2B281F151F192E2802
:100060001E08BE00A8178828281C5A283208073CFA
:10007000031C4028331C051233180516B30C8A28BC
:100080003208083C031C4928A81C0512A8180516AC
:100090008A283208093C031C5328831603130516CB
:1000A000831203138A2832080B3C031C8A28B201EE
:1000B00028108B28B208031D6028051A85288A2875
:1000C0003208083C031C6C28051EB313051AB3172D
:1000D00003198A28B30C8A283208093C031C7128AA
:1000E0008A28051E852828197E28A717831603133A
:1000F00006108312031306100B12862823083302FE
:10010000031D85282811B2018B28B301B2018B2869
:100110000B108C28B20A8B10300884002F088A003C
:100120002E0E8300AD0E2D0E09003308B400F03CF6
:10013000031D9D28A714A711752BA71CF92AA7102A
:100140003308123C0319A7283308593C0319271117
:100150003308583C031DCC28271EBD282712ED303C
:10016000B30034251B25FA30412535113508B3007D
:1001700034251B25FA304125752B2716ED30B300A9
:1001800034251B25FA30412535153508B3003425B3
:100190001B25FA304125752B3308113C031DD2284D
:1001A000A712B62B3308143C031D752B2713ED2B18
:1002E00002309F00831203130910831603130910B1
:1002F0008312031383160313181117309900831206
:1003000003139817831603138C169816831203137E
:100310000B17181683160313061405160113831200
:1003200003130B1683160313051486178312031386
:10033000C1309F008B15F8308B058C018D018B1718
:100340000230B500B201A701A801831603130130E2
:10035000880583120313881208138813E130880577
:10036000043097240330A724C12401309724083097
:10037000A724C124013097240230A724C1240130CE
:1003800097242830AE240C30AE242830AE2401301F
:10039000AE242830B600B7012730A50002308A000D
:1003A0002508273C1B22A60013252608B024A50BF0
:1003B000CE290D3013250A3013250A301325FF30BE
:1003C000B30034251B25ED30B30034251B25FA304E
:1003D00041253508B30034251B25FA304125ED3081
:1003E000B30034251B25FA30412535143508B300F8
:1003F00034251B25FA304125FF30A0000430FC24B1
:1004000080309724FF30A0000430FC24103090246A
:1004100007309E24C830A0000430FC24803097248C
:10042000B430A0000330FC24A71B952027184625D4
:10043000A81B7F25142A82075034493443343134B1
:10044000363446343734373420344134543420344D
:100450004B346534793462346F34613472346434CB
:10046000203442346F3478342034563430342E34CF
:100470003034343420347334743461346E3464343E
:100480002D346234793482074C345A3469347834E8
:1004900087349734A734B834C934DA34EC34FE34B2
:1004A00082072A34373434343134303438343534F4
:0A04B0003234233439343634333447
:1005000082070034393400343534333431343234F2
:1005100032340034303438343634343409347E34B0
:10052000003400347F2B7D2B0034812B7134313427
:100530000034003400347A34733461347734323424
:100540000034003463347834643465343434333400
:1005500000340034203476346634743472343534E4
:10056000003400346E34623468346734793436349D
:100570000034003400346D346A3475343734383420
:10058000003400342C346B3469346F3430343934F3
:10059000003400342E343F346C343B3470342D340A
:1005A000003400340034273400345B342B340034FE
:1005B000003400347D2B6E2B5D3400347C340034E9
:1005C000003400343C3430342E3432343534363454
:1005D00038340034003431342B3433342D342A345D
:1005E000393400340834003400343134373434348E
:1005F0003734A71D0B2BA71A0B2B271B0B2B3308EC
:100600004A3C031D062B2F30B3003F2B33085A3CC6
:1006100003180B2B752B3308613C0318212B0E306C
:10062000B3023308613C031C182B1930B307212B8C
:100630003308773C0318212B3308D23C0319A71544
:10064000752B02308A0033088022B300B3080319E7
:10065000752BA71A992B271B872B3308603C03188F
:10066000062C33087A3C031C062C3308271A3B2B34
:10067000271D3F2B3D2B27193F2BE03EB3003308AE
:1006800013253308083C031D532B37080319752B1A
:10069000B7033708403E8038A500AE242030B02490
:1006A0002508AE24752B3308093C031D602B370841
:1006B000263C031C5E2B2030B024B70A2030B30048
:1006C0003708273C0318662BA816B5253708403E87
:1006D0008038AE243308B024B70A752BA816B52588
:1006E0000D3013250A301325003483160313061426
:1006F00083120313A7130B16080027150034A7163F
:10070000822B2717B801B901BA01BB0100343308A5
:10071000403C0318992B3308463C031C912BB3161D
:10072000A12B3308603C0318992B3308663C03184F
:10073000A12B3308293C0318752B3308393C031CC3
:10074000752BB808031DA82BB80A3308B900752B00
:10075000380BAE2BB80A3308BA00752B3808023CA8
:10076000031D752BB80A3308BB00752BB808031995
:10077000752B3030B902BA02BB02B803031DC32B7C
:100780003908B300DD2BB803031DCD2B03308A00DD
:100790003908DF233A07B300DD2B3908023C031C7C
:1007A000752B03308A0039080A3EDF23B9003A0866
:1007B000DF23B9073B083907B300B8013F2B820795
:1007C00000340A3414341E34283432343C34463471
:1007D00050345A3400346434C834B8080319752BC3
:1007E0003030B902BA02B91EF72B2730B902BA1E4F
:1007F000FB2B2730BA02B803031D012C3908B300C4
:10080000042C390E3A04B300B8013F2B271D3F2BAF
:1008100033080D3C03183F2B3408613C031C3F2B6D
:1008200034083C3C0318172C3D30B402202C34080B
:10083000243C03181E2C2330B402202C0430B407AF
:1008400004308A0034082624B3003F2B8207263464
:100850002A34243423343C34003400340034293422
:100860002834003425343E342F3400343A340034F4
:100870005F3460345E340034223400347B343D34E1
:10088000003421340034003400347D3400345C34CE
:080890000034403400343E3412
:10092000A000810183160313C03081050800A000D8
:10093000810183160313C0308105013081048312C5
:1009400003130B110B1DA22CA00BA12C0800A2005D
:10095000E1308805220D1E39880408002816B12CC4
:100960002812A300C524281E88172308230EA724B5
:10097000C1242308A724C124E13088058813081363
:10098000080088160000881208008813A81583162E
:1009900003131E3088048312031308178816081ED9
:1009A000A81188120000C124A819CE2C08138316A0
:1009B0000313E13088058312031308003C08BD00CF
:1009C00028136430A100EC240A30A100EC2401308B
:1009D000A1002817EC240800A00121083D02031CF7
:1009E000F62CA00A2108BD022817EE2C3030200773
:1009F000281F2030B0240800A100810183160313B2
:100A000007308100831203130B1109140E250910FE
:100A10000E250B1D052DA10B042D08002008A2009A
:100A2000A20B102D080083160313981C152D83129A
:100A30000313990008000B12831603130610051206
:100A400083120313061005122030A000A00B262DE0
:100A5000B2018316031306148312031328148B1098
:100A60000B162818312D0800A2000830A300A4019D
:100A70002218A40AA20CA30B382DA810241CA81419
:100A80000800A30028152819432D08002A08AC00E7
:100A90005A25291C542D2B08AC005A252910981CC6
:100AA000542D181218111816831603138C1683125E
:100AB000031308002C08083C031D682D3608031991
:100AC0007D2DB60336088038AE242030B0247D2D2D
:100AD0003608273C03186E2DA812B5253608803835
:100AE000AE242C080D3C031C7A2D031D7D2DA8126D
:100AF000B5257D2D2C08B024B60A271008003E0825
:100B0000BC00F030A0000430FC24C030AE245630CD
:100B1000B0246130B0246C30B0242030B0243D309B
:100B2000B0242030B024DE242030B0242030B02483
:100B30000B30A50002308A0025084322FD3EA600A6
:100B40003E02031CA82D26083E02063C0318AA2DCF
:100B5000A50B9A2D02308A00250850221325B024B7
:100B60002030B024A8138B1508002830A81AC32DF4
:100B7000B6008030AE242030B024B60BBB2D8030C0
:100B8000AE24B6010800B700C030AE242030B02437
:0C0B9000B70BC62DC030AE24B701080022
:02400E00F23F7F
:00000001FF
